 lcdad

 Timestamp is 4fb05c75 (Mon May 14 13:14:29 2012)

 Preferred load address is 10000000

 Start         Length     Name                   Class
 0001:00000000 00000004H .CRT$XCA                CODE
 0001:00000004 00000004H .CRT$XCZ                CODE
 0001:00000008 00000004H .CRT$XIA                CODE
 0001:0000000c 00000004H .CRT$XIZ                CODE
 0001:00000010 00000004H .CRT$XPA                CODE
 0001:00000014 00000004H .CRT$XPZ                CODE
 0001:00000018 00000004H .CRT$XTA                CODE
 0001:0000001c 00000004H .CRT$XTZ                CODE
 0001:00000020 00000c1cH .rdata                  CODE
 0001:00000c3c 00000022H .rdata$debug            CODE
 0001:00000c60 00001ff4H .text                   CODE
 0001:00002c54 00000028H .xdata                  CODE
 0001:00002c7c 00000028H .idata$2                CODE
 0001:00002ca4 00000014H .idata$3                CODE
 0001:00002cb8 00000088H .idata$4                CODE
 0001:00002d40 0000006eH .idata$6                CODE
 0001:00002db0 000000d8H .edata                  CODE
 0002:00000000 00000088H .idata$5                DATA
 0002:00000088 000004d4H .data                   DATA
 0002:00000560 00000fb8H .bss                    DATA
 0003:00000000 00000148H .pdata                  DATA

  Address         Publics by Value              Rva+Base       Lib:Object

 0000:00000000       ___safe_se_handler_count   00000000     <absolute>
 0000:00000000       ___safe_se_handler_table   00000000     <absolute>
 0001:00000000       __xc_a                     10001000     corelib0:crt0init.obj
 0001:00000004       __xc_z                     10001004     corelib0:crt0init.obj
 0001:00000008       __xi_a                     10001008     corelib0:crt0init.obj
 0001:0000000c       __xi_z                     1000100c     corelib0:crt0init.obj
 0001:00000010       __xp_a                     10001010     corelib0:crt0init.obj
 0001:00000014       __xp_z                     10001014     corelib0:crt0init.obj
 0001:00000018       __xt_a                     10001018     corelib0:crt0init.obj
 0001:0000001c       __xt_z                     1000101c     corelib0:crt0init.obj
 0001:00000040       ??_C@_1FC@MJFNJJFC@?$AAL?$AAC?$AAD?$AA?5?$AAA?$AAu?$AAt?$AAo?$AAd?$AAe?$AAt?$AAe?$AAc?$AAt?$AA?5?$AAD?$AAr?$AAi?$AAv?$AAe?$AAr?$AA?3?$AA?5?$AA?9?$AAD?$AAl?$AAl?$AAM?$AAa?$AAi?$AAn?$AA?$CI@ 10001040     LCDAD.obj
 0001:00000098       ??_C@_1JE@GDGCNPFM@?$AAL?$AAC?$AAD?$AA?5?$AAA?$AAu?$AAt?$AAo?$AAd?$AAe?$AAt?$AAe?$AAc?$AAt?$AA?5?$AAD?$AAr?$AAi?$AAv?$AAe?$AAr?$AA?3?$AA?5?$AA?$CL?$AAD?$AAl?$AAl?$AAM?$AAa?$AAi?$AAn?$AA?$CI@ 10001098     LCDAD.obj
 0001:00000130       ??_C@_1EM@CJFPIJKL@?$AAL?$AAC?$AAD?$AA?5?$AAA?$AAu?$AAt?$AAo?$AAd?$AAe?$AAt?$AAe?$AAc?$AAt?$AA?5?$AAD?$AAr?$AAi?$AAv?$AAe?$AAr?$AA?3?$AA?5?$AA?9?$AAI?$AAn?$AAi?$AAt?$AA?$CI?$AAN?$AAU?$AAL@ 10001130     LCDAD.obj
 0001:0000017c       ??_C@_19OBGHODPD@?$AAM?$AAo?$AAd?$AAe?$AA?$AA@ 1000117c     LCDAD.obj
 0001:00000188       ??_C@_1HC@FJPGMNNN@?$AAL?$AAC?$AAD?$AA?5?$AAA?$AAu?$AAt?$AAo?$AAd?$AAe?$AAt?$AAe?$AAc?$AAt?$AA?5?$AAD?$AAr?$AAi?$AAv?$AAe?$AAr?$AA?3?$AA?5?$AA?$CL?$AAI?$AAn?$AAi?$AAt?$AA?$CI?$AAs?$AAz?$AAA@ 10001188     LCDAD.obj
 0001:00000200       ??_C@_1FA@OBBJIGHP@?$AAL?$AAC?$AAD?$AA?5?$AAA?$AAu?$AAt?$AAo?$AAd?$AAe?$AAt?$AAe?$AAc?$AAt?$AA?5?$AAD?$AAr?$AAi?$AAv?$AAe?$AAr?$AA?3?$AA?5?$AA?9?$AAD?$AAe?$AAi?$AAn?$AAi?$AAt?$AA?$CI?$AAT@ 10001200     LCDAD.obj
 0001:00000250       ??_C@_1EI@OJPAAHMP@?$AAL?$AAC?$AAD?$AA?5?$AAA?$AAu?$AAt?$AAo?$AAd?$AAe?$AAt?$AAe?$AAc?$AAt?$AA?5?$AAD?$AAr?$AAi?$AAv?$AAe?$AAr?$AA?3?$AA?5?$AA?$CL?$AAD?$AAe?$AAi?$AAn?$AAi?$AAt?$AA?$CI?$AA?$CJ@ 10001250     LCDAD.obj
 0001:00000298       ??_C@_1EM@GJKJCLLA@?$AAL?$AAC?$AAD?$AA?5?$AAA?$AAu?$AAt?$AAo?$AAd?$AAe?$AAt?$AAe?$AAc?$AAt?$AA?5?$AAD?$AAr?$AAi?$AAv?$AAe?$AAr?$AA?3?$AA?5?$AA?9?$AAO?$AAp?$AAe?$AAn?$AA?$CI?$AAN?$AAU?$AAL@ 10001298     LCDAD.obj
 0001:000002e8       ??_C@_1EE@BKFDLIJE@?$AAL?$AAC?$AAD?$AA?5?$AAA?$AAu?$AAt?$AAo?$AAd?$AAe?$AAt?$AAe?$AAc?$AAt?$AA?5?$AAD?$AAr?$AAi?$AAv?$AAe?$AAr?$AA?3?$AA?5?$AA?$CL?$AAO?$AAp?$AAe?$AAn?$AA?$CI?$AA?$CJ?$AA?$CL?$AA?$AN@ 100012e8     LCDAD.obj
 0001:00000330       ??_C@_1FA@JFEGFKEB@?$AAL?$AAC?$AAD?$AA?5?$AAA?$AAu?$AAt?$AAo?$AAd?$AAe?$AAt?$AAe?$AAc?$AAt?$AA?5?$AAD?$AAr?$AAi?$AAv?$AAe?$AAr?$AA?3?$AA?5?$AA?9?$AAC?$AAl?$AAo?$AAs?$AAe?$AA?$CI?$AAF?$AAA@ 10001330     LCDAD.obj
 0001:00000380       ??_C@_1EG@NPNPFEIA@?$AAL?$AAC?$AAD?$AA?5?$AAA?$AAu?$AAt?$AAo?$AAd?$AAe?$AAt?$AAe?$AAc?$AAt?$AA?5?$AAD?$AAr?$AAi?$AAv?$AAe?$AAr?$AA?3?$AA?5?$AA?$CL?$AAC?$AAl?$AAo?$AAs?$AAe?$AA?$CI?$AA?$CJ?$AA?$CL@ 10001380     LCDAD.obj
 0001:000003c8       ??_C@_1EI@MILDGJHC@?$AAL?$AAC?$AAD?$AA?5?$AAA?$AAu?$AAt?$AAo?$AAd?$AAe?$AAt?$AAe?$AAc?$AAt?$AA?5?$AAD?$AAr?$AAi?$AAv?$AAe?$AAr?$AA?3?$AA?5?$AA?9?$AAR?$AAe?$AAa?$AAd?$AA?$CI?$AA?9?$AA1?$AA?$CJ@ 100013c8     LCDAD.obj
 0001:00000410       ??_C@_1EE@IAJLLOPP@?$AAL?$AAC?$AAD?$AA?5?$AAA?$AAu?$AAt?$AAo?$AAd?$AAe?$AAt?$AAe?$AAc?$AAt?$AA?5?$AAD?$AAr?$AAi?$AAv?$AAe?$AAr?$AA?3?$AA?5?$AA?$CL?$AAR?$AAe?$AAa?$AAd?$AA?$CI?$AA?$CJ?$AA?$CL?$AA?$AN@ 10001410     LCDAD.obj
 0001:00000458       ??_C@_1EK@EBBLJDD@?$AAL?$AAC?$AAD?$AA?5?$AAA?$AAu?$AAt?$AAo?$AAd?$AAe?$AAt?$AAe?$AAc?$AAt?$AA?5?$AAD?$AAr?$AAi?$AAv?$AAe?$AAr?$AA?3?$AA?5?$AA?9?$AAW?$AAr?$AAi?$AAt?$AAe?$AA?$CI?$AA?9?$AA1@ 10001458     LCDAD.obj
 0001:000004a8       ??_C@_1EG@CADCCJHD@?$AAL?$AAC?$AAD?$AA?5?$AAA?$AAu?$AAt?$AAo?$AAd?$AAe?$AAt?$AAe?$AAc?$AAt?$AA?5?$AAD?$AAr?$AAi?$AAv?$AAe?$AAr?$AA?3?$AA?5?$AA?$CL?$AAW?$AAr?$AAi?$AAt?$AAe?$AA?$CI?$AA?$CJ?$AA?$CL@ 100014a8     LCDAD.obj
 0001:000004f0       ??_C@_1EI@PBAEEDGE@?$AAL?$AAC?$AAD?$AA?5?$AAA?$AAu?$AAt?$AAo?$AAd?$AAe?$AAt?$AAe?$AAc?$AAt?$AA?5?$AAD?$AAr?$AAi?$AAv?$AAe?$AAr?$AA?3?$AA?5?$AA?9?$AAS?$AAe?$AAe?$AAk?$AA?$CI?$AA?9?$AA1?$AA?$CJ@ 100014f0     LCDAD.obj
 0001:00000538       ??_C@_1EE@GHFJHNMI@?$AAL?$AAC?$AAD?$AA?5?$AAA?$AAu?$AAt?$AAo?$AAd?$AAe?$AAt?$AAe?$AAc?$AAt?$AA?5?$AAD?$AAr?$AAi?$AAv?$AAe?$AAr?$AA?3?$AA?5?$AA?$CL?$AAS?$AAe?$AAe?$AAk?$AA?$CI?$AA?$CJ?$AA?$CL?$AA?$AN@ 10001538     LCDAD.obj
 0001:00000580       ??_C@_1FI@NLFIOOA@?$AAL?$AAC?$AAD?$AA?5?$AAA?$AAu?$AAt?$AAo?$AAd?$AAe?$AAt?$AAe?$AAc?$AAt?$AA?5?$AAD?$AAr?$AAi?$AAv?$AAe?$AAr?$AA?3?$AA?5?$AA?9?$AAI?$AAO?$AAC?$AAo?$AAn?$AAt?$AAr?$AAo@ 10001580     LCDAD.obj
 0001:000005d8       ??_C@_1EO@BIJIHCPO@?$AAL?$AAC?$AAD?$AA?5?$AAA?$AAu?$AAt?$AAo?$AAd?$AAe?$AAt?$AAe?$AAc?$AAt?$AA?5?$AAD?$AAr?$AAi?$AAv?$AAe?$AAr?$AA?3?$AA?5?$AA?$CL?$AAI?$AAO?$AAC?$AAo?$AAn?$AAt?$AAr?$AAo@ 100015d8     LCDAD.obj
 0001:000008c0       ??_C@_1LK@EOFGJIPA@?$AAE?$AAR?$AAR?$AAO?$AAR?$AA?3?$AA?5?$AAF?$AAa?$AAi?$AAl?$AAe?$AAd?$AA?5?$AAt?$AAo?$AA?5?$AAw?$AAr?$AAi?$AAt?$AAe?$AA?5?$AA0?$AAx?$AA?$CF?$AA0?$AA2?$AAX?$AA?5?$AAt?$AAo@ 100018c0     lcdeeprom.obj
 0001:00000980       ??_C@_1FG@FMFJNMKP@?$AAE?$AAR?$AAR?$AAO?$AAR?$AA?3?$AA?5?$AAL?$AAC?$AAD?$AA_?$AAM?$AAO?$AAD?$AAE?$AA_?$AAI?$AAN?$AAF?$AAO?$AA?5?$AAt?$AAo?$AAo?$AA?5?$AAb?$AAi?$AAg?$AA?5?$AAf?$AAo?$AAr@ 10001980     lcdeeprom.obj
 0001:000009d8       ??_C@_1KI@JPAGLBFF@?$AAE?$AAR?$AAR?$AAO?$AAR?$AA?3?$AA?5?$AAF?$AAa?$AAi?$AAl?$AAe?$AAd?$AA?5?$AAt?$AAo?$AA?5?$AAr?$AAe?$AAa?$AAd?$AA?5?$AAI?$AA2?$AAC?$AA?5?$AAr?$AAe?$AAg?$AAi?$AAs?$AAt@ 100019d8     lcdeeprom.obj
 0001:00000a80       ??_C@_1FC@NEANMAHD@?$AAE?$AAR?$AAR?$AAO?$AAR?$AA?3?$AA?5?$AAC?$AAa?$AAn?$AA?8?$AAt?$AA?5?$AAo?$AAp?$AAe?$AAn?$AA?5?$AAI?$AA2?$AAC?$AA?5?$AAd?$AAr?$AAi?$AAv?$AAe?$AAr?$AA?$CB?$AA?5?$AA?$CI?$AAE@ 10001a80     lcdeeprom.obj
 0001:00000ad8       ??_C@_1HC@NLFAGOED@?$AAE?$AAR?$AAR?$AAO?$AAR?$AA?3?$AA?5?$AAF?$AAa?$AAi?$AAl?$AAe?$AAd?$AA?5?$AAt?$AAo?$AA?5?$AAs?$AAe?$AAt?$AA?5?$AAI?$AA2?$AAC?$AA?5?$AAf?$AAr?$AAe?$AAq?$AAu?$AAe?$AAn@ 10001ad8     lcdeeprom.obj
 0001:00000b50       ??_C@_1GK@GNNMGJPC@?$AAE?$AAR?$AAR?$AAO?$AAR?$AA?3?$AA?5?$AAF?$AAa?$AAi?$AAl?$AAe?$AAd?$AA?5?$AAt?$AAo?$AA?5?$AAs?$AAe?$AAt?$AA?5?$AAT?$AAo?$AAp?$AAa?$AAz?$AA?5?$AAa?$AAs?$AA?5?$AAI?$AA2@ 10001b50     lcdeeprom.obj
 0001:00000bbc       ??_C@_1M@LCEEOPDH@?$AAI?$AA2?$AAC?$AA1?$AA?3?$AA?$AA@ 10001bbc     lcdeeprom.obj
 0001:00000bc8       ??_C@_1HE@IEHCEBIC@?$AAO?$AAl?$AAd?$AA?5?$AAL?$AAC?$AAD?$AA?5?$AAt?$AAy?$AAp?$AAe?$AA?5?$AAd?$AAa?$AAt?$AAa?$AA?5?$AAf?$AAo?$AAu?$AAn?$AAd?$AA?3?$AA?5?$AA?$CF?$AAd?$AA?4?$AA?5?$AAU?$AAp?$AAg@ 10001bc8     lcdeeprom.obj
 0001:00000c60       ?to_T@@YAPBGPBD@Z          10001c60 f   DebugZones.obj
 0001:00000d00       DllMain                    10001d00 f   LCDAD.obj
 0001:00000db8       ?Init@@YAPAXPAX@Z          10001db8 f   LCDAD.obj
 0001:00000eb0       ?Deinit@@YAHPAX@Z          10001eb0 f   LCDAD.obj
 0001:00000f3c       ?Open@@YAPAXPAXKK@Z        10001f3c f   LCDAD.obj
 0001:00000fc8       ?Close@@YAHPAX@Z           10001fc8 f   LCDAD.obj
 0001:00001054       ?Read@@YAKPAXPAEK@Z        10002054 f   LCDAD.obj
 0001:000010e0       ?Write@@YAKPAXPAEK@Z       100020e0 f   LCDAD.obj
 0001:0000116c       ?Seek@@YAKPAXJK@Z          1000216c f   LCDAD.obj
 0001:000011f8       ?IOControl@@YAHPAXKPAEK1KPAK@Z 100021f8 f   LCDAD.obj
 0001:00001284       ?PowerUp@@YAHPAX@Z         10002284 f   LCDAD.obj
 0001:000012ac       ?PowerDown@@YAHPAX@Z       100022ac f   LCDAD.obj
 0001:000012d4       ?WriteI2CRegister@@YAHPAXEEE@Z 100022d4 f   lcdeeprom.obj
 0001:000013c0       ?WriteI2CRegister@@YAHPAXEGE@Z 100023c0 f   lcdeeprom.obj
 0001:000014c4       ?GetModeFromEEPROM@@YAPAULCD_MODE_INFO@@XZ 100024c4 f   lcdeeprom.obj
 0001:00002208       RegisterDbgZones           10003208 f   coredll:COREDLL.dll
 0001:00002218       DisableThreadLibraryCalls  10003218 f   coredll:COREDLL.dll
 0001:00002228       NKDbgPrintfW               10003228 f   coredll:COREDLL.dll
 0001:00002238       RegCloseKey                10003238 f   coredll:COREDLL.dll
 0001:00002248       RegSetValueExW             10003248 f   coredll:COREDLL.dll
 0001:00002258       OpenDeviceKey              10003258 f   coredll:COREDLL.dll
 0001:00002268       GetLastError               10003268 f   coredll:COREDLL.dll
 0001:00002278       Sleep                      10003278 f   coredll:COREDLL.dll
 0001:00002288       I2CTransfer                10003288 f   i2csdk:I2CSDK.dll
 0001:00002298       I2CCloseHandle             10003298 f   i2csdk:I2CSDK.dll
 0001:000022a8       I2CSetFrequency            100032a8 f   i2csdk:I2CSDK.dll
 0001:000022b8       I2CSetMasterMode           100032b8 f   i2csdk:I2CSDK.dll
 0001:000022c8       I2COpenHandle              100032c8 f   i2csdk:I2CSDK.dll
 0001:000022d8       _DllMainCRTStartup         100032d8 f   corelib0:pegdmain.obj
 0001:00002480       __security_init_cookie     10003480 f   corelib0:seccinit.obj
 0001:00002548       exit                       10003548 f   corelib0:cexit.obj
 0001:000026c8       _exit                      100036c8 f   corelib0:cexit.obj
 0001:000026ec       _cexit                     100036ec f   corelib0:cexit.obj
 0001:00002708       _c_exit                    10003708 f   corelib0:cexit.obj
 0001:00002724       GetCurrentProcess          10003724 f i corelib0:cexit.obj
 0001:0000273c       _initterm                  1000373c f   corelib0:crt0dat.obj
 0001:00002790       _cinit                     10003790 f   corelib0:crt0dat.obj
 0001:000027cc       _onexit                    100037cc f   corelib0:onexit.obj
 0001:00002ad0       atexit                     10003ad0 f   corelib0:onexit.obj
 0001:00002b24       mbstowcs                   10003b24 f   corelib1:COREDLL.dll
 0001:00002b34       memcmp                     10003b34 f   corelib1:COREDLL.dll
 0001:00002b44       memcpy                     10003b44 f   corelib1:COREDLL.dll
 0001:00002b54       __rt_sdiv                  10003b54 f   corelib1:COREDLL.dll
 0001:00002b64       memset                     10003b64 f   corelib1:COREDLL.dll
 0001:00002b74       _XcptFilter                10003b74 f   corelib1:COREDLL.dll
 0001:00002b84       __C_specific_handler       10003b84 f   corelib1:COREDLL.dll
 0001:00002b94       __security_gen_cookie2     10003b94 f   corelib1:COREDLL.dll
 0001:00002ba4       free                       10003ba4 f   corelib1:COREDLL.dll
 0001:00002bb4       malloc                     10003bb4 f   corelib1:COREDLL.dll
 0001:00002bc4       realloc                    10003bc4 f   corelib1:COREDLL.dll
 0001:00002bd4       _msize                     10003bd4 f   corelib1:COREDLL.dll
 0001:00002be4       DeleteCriticalSection      10003be4 f   coredll:COREDLL.dll
 0001:00002bf4       InterlockedExchange        10003bf4 f   coredll:COREDLL.dll
 0001:00002c04       TerminateProcess           10003c04 f   coredll:COREDLL.dll
 0001:00002c14       EnterCriticalSection       10003c14 f   coredll:COREDLL.dll
 0001:00002c24       InterlockedCompareExchange 10003c24 f   coredll:COREDLL.dll
 0001:00002c34       InitializeCriticalSection  10003c34 f   coredll:COREDLL.dll
 0001:00002c44       LeaveCriticalSection       10003c44 f   coredll:COREDLL.dll
 0001:00002c7c       __IMPORT_DESCRIPTOR_COREDLL 10003c7c     coredll:COREDLL.dll
 0001:00002c90       __IMPORT_DESCRIPTOR_I2CSDK 10003c90     i2csdk:I2CSDK.dll
 0001:00002ca4       __NULL_IMPORT_DESCRIPTOR   10003ca4     coredll:COREDLL.dll
 0002:00000000       __imp_RegisterDbgZones     10004000     coredll:COREDLL.dll
 0002:00000004       __imp_DisableThreadLibraryCalls 10004004     coredll:COREDLL.dll
 0002:00000008       __imp_NKDbgPrintfW         10004008     coredll:COREDLL.dll
 0002:0000000c       __imp_RegCloseKey          1000400c     coredll:COREDLL.dll
 0002:00000010       __imp_RegSetValueExW       10004010     coredll:COREDLL.dll
 0002:00000014       __imp_OpenDeviceKey        10004014     coredll:COREDLL.dll
 0002:00000018       __imp_GetLastError         10004018     coredll:COREDLL.dll
 0002:0000001c       __imp_Sleep                1000401c     coredll:COREDLL.dll
 0002:00000020       __imp_InitializeCriticalSection 10004020     coredll:COREDLL.dll
 0002:00000024       __imp_InterlockedCompareExchange 10004024     coredll:COREDLL.dll
 0002:00000028       __imp_EnterCriticalSection 10004028     coredll:COREDLL.dll
 0002:0000002c       __imp_TerminateProcess     1000402c     coredll:COREDLL.dll
 0002:00000030       __imp_InterlockedExchange  10004030     coredll:COREDLL.dll
 0002:00000034       __imp_DeleteCriticalSection 10004034     coredll:COREDLL.dll
 0002:00000038       __imp_mbstowcs             10004038     corelib1:COREDLL.dll
 0002:0000003c       __imp_memcmp               1000403c     corelib1:COREDLL.dll
 0002:00000040       __imp_memcpy               10004040     corelib1:COREDLL.dll
 0002:00000044       __imp___rt_sdiv            10004044     corelib1:COREDLL.dll
 0002:00000048       __imp_memset               10004048     corelib1:COREDLL.dll
 0002:0000004c       __imp__XcptFilter          1000404c     corelib1:COREDLL.dll
 0002:00000050       __imp___C_specific_handler 10004050     corelib1:COREDLL.dll
 0002:00000054       __imp___security_gen_cookie2 10004054     corelib1:COREDLL.dll
 0002:00000058       __imp_free                 10004058     corelib1:COREDLL.dll
 0002:0000005c       __imp_malloc               1000405c     corelib1:COREDLL.dll
 0002:00000060       __imp_realloc              10004060     corelib1:COREDLL.dll
 0002:00000064       __imp__msize               10004064     corelib1:COREDLL.dll
 0002:00000068       __imp_LeaveCriticalSection 10004068     coredll:COREDLL.dll
 0002:0000006c       \177COREDLL_NULL_THUNK_DATA 1000406c     coredll:COREDLL.dll
 0002:00000070       __imp_I2CSetMasterMode     10004070     i2csdk:I2CSDK.dll
 0002:00000074       __imp_I2CSetFrequency      10004074     i2csdk:I2CSDK.dll
 0002:00000078       __imp_I2CCloseHandle       10004078     i2csdk:I2CSDK.dll
 0002:0000007c       __imp_I2CTransfer          1000407c     i2csdk:I2CSDK.dll
 0002:00000080       __imp_I2COpenHandle        10004080     i2csdk:I2CSDK.dll
 0002:00000084       \177I2CSDK_NULL_THUNK_DATA 10004084     i2csdk:I2CSDK.dll
 0002:00000088       dpCurSettings              10004088     DebugZones.obj
 0002:00000554       __security_cookie          10004554     corelib0:seccinit.obj
 0002:00000558       __security_cookie_complement 10004558     corelib0:seccinit.obj
 0002:00001504       _exitflag                  10005504     corelib0:cexit.obj
 0002:00001508       __onexitend                10005508     <common>
 0002:0000150c       __onexitbegin              1000550c     <common>
 0002:00001510       g_pcsExit                  10005510     <common>
 0002:00001514       _pRawDllMain               10005514     <common>

 entry point at        0001:000022d8

 Static symbols

 0001:0000184c       ?ReadI2CRegister@@YAHPAXEEPAEG@Z 1000284c f   lcdeeprom.obj
 0001:0000193c       ?ReadI2CRegister@@YAHPAXEGPAEG@Z 1000293c f   lcdeeprom.obj
 0001:00001a4c       ?SetupI2C@@YAPAXK@Z        10002a4c f   lcdeeprom.obj
 0001:00001b64       ?DetectEEPROM@@YA?AW4EEPROM_TYPE@@PAX@Z 10002b64 f   lcdeeprom.obj
 0001:00001c90       ?GetPanelType@@YAKPAX@Z    10002c90 f   lcdeeprom.obj
 0001:00001d90       ?IsValidPanelType@@YAHK@Z  10002d90 f   lcdeeprom.obj
 0001:00001e60       ?WriteMode@@YAXPAXK@Z      10002e60 f   lcdeeprom.obj
 0001:00002068       ?WriteMode32@@YAXPAXK@Z    10003068 f   lcdeeprom.obj
 0001:0000232c       _DllMainCRTStartupHelper   1000332c f   corelib0:pegdmain.obj
 0001:0000256c       doexit                     1000356c f   corelib0:cexit.obj
 0001:00002828       lockexit                   10003828 f   corelib0:onexit.obj
 0001:000028c4       unlockexit                 100038c4 f   corelib0:onexit.obj
 0001:000028f0       _onexit_nolock             100038f0 f   corelib0:onexit.obj
